:020000040000FA
:100000000A128A114D2800001830A0000310A70D15
:10001000A80DA90D0310A10DA20DA30D031C1A28F4
:100020002408A70725080318250FA8072608031882
:10003000260FA907A00B062808001830A000A4016D
:10004000A501A6010310AA0DAB0DAC0D0310A10D67
:10005000A20DA30DA40DA50DA60D2708A402280826
:10006000031C280FA5022908031C290FA602031848
:1000700044282708A40728080318280FA5072908DB
:100080000318290FA607031C2A14A00B2228080016
:100090008000840AA00B48280800831330308400B5
:1000A0004E30A000030148208313A030840020308C
:1000B0008312A00003018A1148208A11AE288312FE
:1000C000F300F030831605058312F4000F3073053A
:1000D000F500740875048316850008008312F30088
:1000E0000F30831606058312F4000F307305F500F8
:1000F0000310750DF6000330A2000310F60DA20BDD
:100100007D28740876048316860008003008850070
:1001100008003108860008008312FC00F03030052A
:100120008316BB000F3083127C058316BC003B088E
:100130003C048312B00086288312F6000F3031058C
:10014000F7000310760DF8000330A2000310F80D3D
:10015000A20BA62877087804B10089288312AD0184
:100160006C103229FC00FD01C428831203131630E1
:10017000A2002C30A3000A128A11A30BBB280A127A
:100180008A11A20BB928FD0A7D087C02031DB5283F
:100190000800F701F801E32883120313F230A200EC
:1001A0000A30A3002830A4000A128A11A40BD42814
:1001B0000A128A11A30BD2280A128A11A20BD02884
:1001C000F70A0319F80A78087602031DE928770868
:1001D0007502031DCC2808008316BB003B089B005A
:1001E0001C141A08BC003C080800F30074088316AD
:1001F0009A008312730883169B001C158B138B13B4
:1002000055309D00AA309D009C14000000008B1703
:100210001C119C18092908004030831699001811F8
:1002200008000C2183168C120C1298169030831241
:10023000980008008312FA006C1822290C1E1E294F
:100240007A089900080083128C1E29291A08F300E5
:100250002B2922103029981C2F2918121816221425
:100260007308080011218A113E29B1133108860054
:1002700083168613080083160617080035218A1195
:100280003B2144308312AE00AF0107309F008A113A
:100290006529F600F70150297608B2208312F70A83
:1002A0000A3077028A11031D4C290800F300F4017B
:1002B0005F297308F500F601C9208312F40A0A3099
:1002C00074028A11031D5929080003305621003099
:1002D0008A115F2000308A116E2083160512831266
:1002E00030163008850083160614861185160030F6
:1002F0008A118C2000308A119C2001308312B400B6
:100300000130B5000130B700B8016C120A30DF00CF
:100310000A30E0001430E1000130E2000130E30077
:100320000A30E4001E30E7003230E8008A153F2929
:10033000F6000F30F605F70101307602031DA529FE
:100340000330F6000130F700E72903307602031D81
:10035000AE290630F6000230F700E72902307602B7
:10036000031DB7290630F6000130F700E7290630F3
:100370007602031DC0290C30F6000230F700E72991
:1003800004307602031DC9290C30F6000130F70055
:10039000E7290C307602031DD2290930F60002301D
:1003A000F700E72908307602031DDB290930F60043
:1003B0000130F700E72909307602031DE4290330F4
:1003C000F6000230F700E7290330F600F70176085F
:1003D0000800F6000F30F605F70108307602031D1D
:1003E000F6290C30F6000130F700392A0C3076027D
:1003F000031DFF290630F6000230F700392A0430C9
:100400007602031D082A0630F6000130F700392A6B
:1004100006307602031D112A0330F6000230F70081
:10042000392A02307602031D1A2A0330F600013001
:10043000F700392A03307602031D232A0930F6001B
:100440000230F700392A01307602031D2C2A0930C8
:10045000F6000130F700392A09307602031D352AEB
:100460000C30F6000230F700392A0C30F60002306A
:10047000F70076080800FC000130FD000F30FC0595
:1004800001307C02031D472A0330FC007F2A033021
:100490007C02031D4E2A0230FC007F2A02307C02BF
:1004A000031D552A0630FC007F2A06307C02031DFE
:1004B0005C2A0430FC007F2A04307C02031D632A7E
:1004C0000C30FC007F2A0C307C02031D6A2A0830A5
:1004D000FC007F2A08307C02031D712A0930FC00D1
:1004E0007F2AA20103302202031D782AE9307C0210
:1004F000031D7D2A0130FC007F2A0130FC007C08AE
:100500000800FC000130FD000F30FC0508307C02C3
:10051000031D8D2A0C30FC00C02A0C307C02031D08
:10052000942A0430FC00C02A04307C02031D9B2A5C
:100530000630FC00C02A06307C02031DA22A0230CD
:10054000FC00C02A02307C02031DA92A0330FC00F3
:10055000C02A03307C02031DB02A0130FC00C02AEF
:1005600001307C02031DB72A0930FC00C02A093083
:100570007C02031DBE2A0830FC00C02A0830FC00A3
:100580007C0808003408E9218312B4007708B3001E
:1005900034088A118C2083125F088A11B2208312DA
:1005A0003308B7070030A30023080318230FB80748
:1005B0000800340898218312B4007708B300340887
:1005C0008A118C2083123308B702A2012208031C6F
:1005D000220FB8025F088A11B228350898218312C9
:1005E000B5007708B30035088A119C2083123308C0
:1005F000BB02A2012208031C220FBC022208031C1A
:10060000220FBD0260088A11B2283508E921831241
:10061000B5007708B30035088A119C20831233088F
:10062000BB070030A30023080318230FBC072308CF
:100630000318230FBD0760088A11B22834088122ED
:100640008312B4007D08B30034088A118C20831211
:100650003308B7070030A30023080318230FB80797
:100660005F088A11B22834083B228312B4007D0847
:10067000B30034088A118C2083123308B702A20118
:100680002208031C220FB8025F088A11B22835081D
:100690003B228312B5007D08B30035088A119C20E7
:1006A00083123308BB02A2012208031C220FBC02E2
:1006B0002208031C220FBD0260088A11B2283508E7
:1006C00081228312B5007D08B30035088A119C2071
:1006D00083123308BB070030A30023080318230F3D
:1006E000BC0723080318230FBD0760088A11B2282E
:1006F00020301A213A308A111A21A0308312A70023
:100700008630A8000130A9007708A1007808A2006F
:100710007908A3008A111D2083122A088316BB00C2
:1007200083122B088316BC0083122C088316BD008D
:1007300030303B07BE000030BF0003183F0F3C07BE
:10074000BF000030C0000318400F3C07C0003E0847
:100750008A111A21A0308312A7008630A800013028
:10076000A9007708A1007808A2007908A3008A11DF
:100770001D20831224088316BB00831225088316CC
:10078000BC00831226088316BD0010308312A70018
:100790002730A800A90183163B088312A100831605
:1007A0003C088312A20083163D088312A3008A111D
:1007B0001D2083122A088316BE0083122B0883167D
:1007C000BF0083122C088316C00030303E07C100E2
:1007D0000030C2000318420F3F07C2000030C300C0
:1007E0000318430F3F07C30041088A111A21103034
:1007F0008312A7002730A800A9017708A100780874
:10080000A2007908A3008A111D20831224088316F0
:10081000BB00831225088316BC00831226088316AA
:10082000BD00E8308312A7000330A800A901831699
:100830003B088312A10083163C088312A200831692
:100840003D088312A3008A111D2083122A088316F3
:10085000BE0083122B088316BF0083122C08831658
:10086000C00030303E07C1000030C2000318420F04
:100870003F07C2000030C3000318430F3F07C30007
:1008800041088A111A21E8308312A7000330A8001A
:10089000A9017708A1007808A2007908A3008A11AD
:1008A0001D20831224088316BB008312250883169B
:1008B000BC00831226088316BD0064308312A70093
:1008C000A801A90183163B088312A10083163C08E6
:1008D0008312A20083163D088312A3008A111D20F3
:1008E00083122A088316BE0083122B088316BF00CA
:1008F00083122C088316C00030303E07C100003040
:10090000C2000318420F3F07C2000030C3000318A3
:10091000430F3F07C30041088A111A216430831234
:10092000A700A801A9017708A1007808A20079080A
:10093000A3008A111D20831224088316BB00831292
:1009400025088316BC00831226088316BD000A30D2
:100950008312A700A801A90183163B088312A100F6
:1009600083163C088312A20083163D088312A3005D
:100970008A111D2083122A088316BE0083122B08B9
:100980008316BF0083122C088316C00030303E0748
:10099000C1000030C2000318420F3F07C200003000
:1009A000C3000318430F3F07C30041088A111A21EF
:1009B0000A308312A700A801A9017708A1007808CE
:1009C000A2007908A3008A111D208312240883162F
:1009D000BB00831225088316BC00831226088316E9
:1009E000BD0030303B07BE000030BF0003183F0F92
:1009F0003C07BF000030C0000318400F3C07C00098
:100A00003E088A111A212A308A111A210D308A11C2
:100A10001A210A308A111A298312F300F4012A30AC
:100A20001A218312F5018A11222D47308400831385
:100A30007408840730300007F60076081A21831204
:100A4000F40AF50A750873028A11031D152D0D307D
:100A50001A210A308A111A298312F60014307602FC
:100A6000031D482D41301A2120308A111A2170307F
:100A70008A111A216F308A111A2173308A111A21B2
:100A800083123708F7003808F800F9018A11782333
:100A90001530831276028A11031D652D52301A21FA
:100AA00020308A111A2170308A111A216F308A1170
:100AB0001A2173308A111A2183123B08F7003C086F
:100AC000F8003D08F9008A11782316308312760267
:100AD0008A11031D892D31301A2131308A111A21D2
:100AE0002E308A111A2141308A111A2120308A11A0
:100AF0001A2164308A111A2165308A111A216C304A
:100B00008A111A2183125F08F700F801F9018A118E
:100B100078231730831276028A11031DAD2D3130F0
:100B20001A2132308A111A212E308A111A2152309C
:100B30008A111A2120308A111A2164308A111A214F
:100B400065308A111A216C308A111A2183126008CB
:100B5000F700F801F9018A11782318308312760220
:100B60008A11031DD12D31301A2133308A111A21F7
:100B70002E308A111A2150308A111A2120308A1100
:100B80001A2164308A111A2165308A111A216C30B9
:100B90008A111A2183126108F700F801F9018A11FC
:100BA00078231930831276028A11031DF52D313016
:100BB0001A2134308A111A212E308A111A2141301B
:100BC0008A111A2120308A111A2166308A111A21BD
:100BD00063308A111A2174308A111A218312620833
:100BE000F700F801F9018A1178231A30831276028E
:100BF0008A11031D192E31301A2135308A111A211C
:100C00002E308A111A2152308A111A2120308A116D
:100C10001A2166308A111A2163308A111A21743020
:100C20008A111A2183126308F700F801F9018A1169
:100C300078231B30831276028A11031D402E313037
:100C40001A2136308A111A212E308A111A21503079
:100C50008A111A2120308A111A2144308A111A214E
:100C600069308A111A2173308A111A2174308A115D
:100C70001A2183126808F700F801F9018A11782314
:100C80001C30831276028A11031D642E31301A2122
:100C900037308A111A212E308A111A2150308A11C8
:100CA0001A2120308A111A2164308A111A216930E0
:100CB0008A111A2161308A111A2183126708F700FC
:100CC000F801F9018A1178231D30831276028A1106
:100CD000031D8E2E31301A2138308A111A212E3000
:100CE0008A111A214D308A111A2161308A111A2174
:100CF00078308A111A2120308A111A2164308A1121
:100D00001A2165308A111A2176308A111A2183122C
:100D10006408F700F801F9018A1178231E30831264
:100D200076028A11031DAF2E41301A2163308A11D9
:100D30001A2174308A111A2120308A111A21443064
:100D40008A111A2165308A111A2176308A111A21E6
:100D500083126508F700F801F9018A1178231F3022
:100D6000831276028A11031DC42E56301A212030B8
:100D70008A111A2120308A111A210A308312F700B1
:100D8000F801F9018A1178232030831276028A1142
:100D9000031DEF2E44301A2145308A111A21563096
:100DA0008A111A2149308A111A2141308A111A21D7
:100DB00054308A111A214F308A111A214E308A116B
:100DC0001A2120308A111A2120308A111A21831207
:100DD0006508F7006608F800F9018A11782B080009
:100DE0000130EC208312DF0002308A11EC208312E4
:100DF000E00003308A11EC208312E10004308A11F4
:100E0000EC208312E20005308A11EC208312E3000B
:100E100006308A11EC208312E80007308A11EC209A
:100E20008312E70008308A11EC208312E4001E30A0
:100E30005F027C108A1103191F2F03187C140530E0
:100E40005F02FC100319262F031CFC147C117C1C70
:100E5000FC187C157C1D2E2F0F30DF001E30600229
:100E6000FC110319352F0318FC15053060027C12A4
:100E700003193C2F031C7C16FC12FC1D7C1AFC166B
:100E8000FC1E442F0F30E000C830610203194C2FC4
:100E9000031C4C2F3230E100033062020319542F3F
:100EA000031C542F0130E2000330630203195C2F4E
:100EB000031C5C2F0130E3001E3064020319642F11
:100EC000031C642F0A30E400C830680203196C2F39
:100ED000031C6C2F0A30E800C83067020319742F16
:100EE000031C742F0A30E7000800F0268312F60175
:100EF0008A11892F34083B228312B4007D08B30085
:100F000034088A118C2083125F088A11B220831260
:100F1000F60A0A3076028A11031D7A2F8312061808
:100F2000A02F34083B228312B4007D08B30034089C
:100F30008A118C2083125F088A11B2208A118E2FA9
:100F4000F701B12F340881228312B4007D08B30069
:100F500034088A118C2083125F088A11B220831210
:100F6000F70A323077028A11031DA22F0130B70031
:100F7000B8010618CE2F340881228312B4007D08F0
:100F8000B30034088A118C2083125F088A11B220C2
:100F90008312B70A0319B80A8A11B92FF801DF2F93
:100FA00034083B228312B4007D08B30034088A1150
:100FB0008C2001308312B702031CB802F80A0A30F1
:100FC00078028A11031DD02FEC11F9018A150C2823
:100FD000340881228312B4007D08B30034088A11DA
:100FE0008C2083125F088A11B2208312B70A03197A
:100FF000B80AFA16061CFA127A17EC197A13FA17BD
:10100000FA1A7A1FFA138A15FA1F0B283708C1003B
:101010003808C200EC15F90A143079028A11031D50
:10102000E82F080083127514061C75100301EC19D3
:101030000130A200030175180130A3002208230229
:101040000319592838084202031D2828370841028D
:1010500003193B2803183B283708A2003808A300CF
:101060004108A2024208031C420FA3022208E50025
:101070002308E60049284108A2004208A3003708D7
:10108000A2023808031C380FA3022208E500230837
:10109000E600A20166082202031D502865086402CA
:1010A000031959280318592820308A112C258A1130
:1010B00075278312EC15751CEC1108008312B1150D
:1010C0003108860061088A11492183128A15851A20
:1010D0006528B1113108860001308A114929851E21
:1010E00072285E20831238083A028A15031D7A2876
:1010F000370839020319C62838083A02031D822826
:101100003708390203199E28031C9E28063037072A
:10111000F3000030031801303807F40074083A0275
:10112000031D94287308390203199C2803189C286E
:101130008A111E238A159E288A11C222831238081A
:101140003A028A15031DA628370839020319C22856
:101150000318C22806303907F300003003180130A5
:101160003A07F40038087402031DB82837087302E0
:101170000319C0280318C0288A11D9228A15C22849
:101180008A1133238A1512208A1572280800851EB9
:10119000CA285E2083123D0840028A15031DD62806
:1011A0003C083F02031DD6283B083E0203193E2996
:1011B0003D084002031DE2283C083F02031DE228CF
:1011C0003B083E0203190929031C092906303B0785
:1011D000F3000030F4000318740F3C07F4000030F3
:1011E000F5000318750F3C07F50075084002031D54
:1011F000FF2874083F02031DFF2873083E020319ED
:101200000729031807298A115F238A1509298A11DA
:10121000052383123D0840028A15031D15293C0849
:101220003F02031D15293B083E0203193C29031800
:101230003C2906303E07F3000030F4000318740F19
:101240003F07F4000030F5000318750F3F07F50065
:101250003D087502031D32293C087402031D322922
:101260003B08730203193A2903183A298A11ED221F
:101270008A15CA288A1147238A15CA280800061821
:101280003F29851E44295E208A117527013083126B
:10129000B900BA018A156F20831230123008850018
:1012A00001308A11B2208A1123218312B200EC1777
:1012B000221CEC138A15EC1F922F24303202031DDE
:1012C0006329B601EC1423303202031D6929B601EB
:1012D0006C156D11EC1C6C196D156D1D782947305E
:1012E0008400831336088407D03032078000B60AA2
:1012F00036080B3CED110319ED156D166C19ED1D3B
:101300006D126D1E9B2C3016300885006C11B601D5
:101310004908A100A201A301E830A4000330A50000
:10132000A6018A110420831227088316A0008312C5
:1013300028088316A100831229088316A2008312AD
:101340004A08A100A201A3016430A400A501A601DE
:101350008A110420831227088316A3008312280809
:101360008316A400831229088316A5002008A6006E
:101370002108A7002208A8002308A60724080318AC
:10138000240FA70725080318250FA80783124B0869
:10139000A100A201A3010A30A400A501A6018A119F
:1013A0000420831227088316A900831228088316B5
:1013B000AA00831229088316AB002608AC00270870
:1013C000AD002808AE002908AC072A0803182A0F28
:1013D000AD072B0803182B0FAE072C088312C30090
:1013E00083162D088312C4004C08C3070030A300E5
:1013F00023080318230FC4074E08A100A201A3016C
:10140000E830A4000330A500A6018A11042083124D
:1014100027088316A000831228088316A1008312D0
:1014200029088316A20083124F08A100A201A3017C
:101430006430A400A501A6018A11042083122708A4
:101440008316A300831228088316A4008312290898
:101450008316A5002008A6002108A7002208A800DE
:101460002308A60724080318240FA7072508031834
:10147000250FA80783125008A100A201A3010A307A
:10148000A400A501A6018A1104208312270883164F
:10149000A900831228088316AA008312290883163C
:1014A000AB002608AC002708AD002808AE002908CC
:1014B000AC072A0803182A0FAD072B0803182B0FB7
:1014C000AE072C088312C50083162D088312C600B0
:1014D0005108C5070030A30023080318230FC607CF
:1014E0000B308A110C250030831244028A15031D2B
:1014F0007B2A01304302031D9C2A4508A1004608AF
:10150000A200A3016208A400A501A6018A1104207B
:1015100083122708C5002808C6003708B900380814
:10152000BA004508B90746080318460FBA078A15D6
:101530006F2014308A112C250030831244028A1542
:10154000031DA42A02304302031DD72A4508A10027
:101550004608A200A3016208A400A501A6018A1101
:10156000042083122708C5002808C6003808460250
:101570008A15031DBD2A370845020319D02A03180E
:10158000D02A3708A2003808A3004508A20246085E
:10159000031C460FA3022208B9002308BA00D32A6D
:1015A0000130B900BA016F2014308A112C250030A7
:1015B000831244028A15031DDF2A03304302031DF0
:1015C000082B4508A1004608A200A3016308A40057
:1015D000A501A6018A11042083122708C500280846
:1015E000C6003B08BE003C08BF003D08C0004508DF
:1015F000BE0746080318460FBF070030A3002308A4
:101600000318230FC0078A15C72015308A112C250F
:101610000030831244028A15031D102B043043024C
:10162000031D192B0130B900BA016F2014308A1143
:101630002C250030831244028A15031D212B05300E
:101640004302031D2B2B4108B9004208BA006F204A
:1016500014308A112C250030831244028A15031D90
:10166000332B06304302031D362B5E2000308312DD
:1016700044028A15031D3E2B07304302031D802BB5
:101680004508A1004608A200A3016308A400A50123
:10169000A6018A11042083122708C5002808C60065
:1016A000A2013D0822028A15031D5C2B3C0846025C
:1016B000031D5C2B3B0845020319782B0318782B7C
:1016C0003B08A2003C08A3003D08A4004508A20274
:1016D0004608031C460FA302A5012508031C250F7D
:1016E000A4022208BE002308BF002408C0007C2BEF
:1016F0000130BE00BF01C001C72015308A112C2562
:101700000030831244028A15031D882B08304302DF
:10171000031D902BBB01BC01BD0115308A112C2586
:101720000030831244028A15031D982B09304302AE
:10173000031DAF2B4508A1004608A200A3010A30F3
:10174000A400A501A6018A11042083122708BB006A
:101750002808BC002908BD0015308A112C2500304E
:10176000831244028A15031DB72B0A304302031D5E
:10177000C12B6C1ABD2B6C16BE2B6C1220308A113B
:101780002C250030831244028A15031DC92B0B300F
:101790004302031DD52B4508F40001308A11F520C2
:1017A0008A11F02616308A112C250030831244024B
:1017B0008A15031DDD2B0C304302031DE92B450860
:1017C000F40002308A11F5208A11F02617308A11B0
:1017D0002C250030831244028A15031DF12B0D3095
:1017E0004302031DFD2B4508F40003308A11F52048
:1017F0008A11F02618308A112C25003083124402F9
:101800008A15031D052C0E304302031D112C4508BB
:10181000F40004308A11F5208A11F02619308A115B
:101820002C250030831244028A15031D192C0F3019
:101830004302031D252C4508F40005308A11F520CC
:101840008A11F0261A308A112C25003083124402A6
:101850008A15031D2D2C10304302031D392C450819
:10186000F40006308A11F5208A11F0261B308A1107
:101870002C250030831244028A15031D412C11309F
:101880004302031D4D2C4508F40007308A11F52052
:101890008A11F0261C308A112C2500308312440254
:1018A0008A15031D552C12304302031D612C450877
:1018B000F40008308A11F5208A11F0261D308A11B3
:1018C0002C250030831244028A15031D692C1D301B
:1018D0004302031D712C8A11752714308312C30033
:1018E000C401003044028A15031D782C14304302D1
:1018F000031D8D2C8A11F0268312F2018A15882C83
:1019000043088A112C258312C30A0319C40AF20A58
:101910000C3072028A15031D802C00304402031D16
:10192000932C15304302031D982C1F308A112C254F
:101930008312C301C4013608153C701303197017D4
:10194000F017EC18701FF0138A15F01F922F301645
:1019500030088500EC10B6014908A100A201A301DE
:10196000E830A4000330A500A6018A1104208312E8
:1019700027088316A000831228088316A10083126B
:1019800029088316A20083124A08A100A201A3011C
:101990006430A400A501A6018A110420831227083F
:1019A0008316A300831228088316A4008312290833
:1019B0008316A5002008A6002108A7002208A80079
:1019C0002308A60724080318240FA70725080318CF
:1019D000250FA80783124B08A100A201A3010A301A
:1019E000A400A501A6018A110420831227088316EA
:1019F000A900831228088316AA00831229088316D7
:101A0000AB002608AC002708AD002808AE00290866
:101A1000AC072A0803182A0FAD072B0803182B0F51
:101A2000AE072C088312B90083162D088312BA0062
:101A30004C08B9070030A30023080318230FBA0786
:101A40003908A1003A08A200A3016208A400A50178
:101A5000A6018A11042083122708B9002808BA00B9
:101A60008A156F2015308A110C2583124E08A100AB
:101A7000A201A301A030A4008630A5000130A60079
:101A80008A110420831227088316A00083122808D5
:101A90008316A100831229088316A20083124F081F
:101AA000A100A201A3011030A4002730A500A601C7
:101AB0008A110420831227088316A30083122808A2
:101AC0008316A400831229088316A5002008A60007
:101AD0002108A7002208A8002308A6072408031845
:101AE000240FA70725080318250FA80783125008FD
:101AF000A100A201A301E830A4000330A500A601C3
:101B00008A110420831227088316A900831228084B
:101B10008316AA00831229088316AB002608AC009E
:101B20002708AD002808AE002908AC072A080318CA
:101B30002A0FAD072B0803182B0FAE07831251088D
:101B4000A100A201A3016430A400A501A6018A118D
:101B50000420831227088316AF00831228088316F7
:101B6000B000831229088316B1002C08B2002D089A
:101B7000B3002E08B4002F08B20730080318300F46
:101B8000B30731080318310FB40783125208A100BC
:101B9000A201A3010A30A400A501A6018A11042014
:101BA000831227088316B500831228088316B6000F
:101BB000831229088316B7003208B8003308B90029
:101BC0003408BA003508B80736080318360FB907C5
:101BD00037080318370FBA0738088312BE00831678
:101BE00039088312BF0083163A088312C0005308D5
:101BF000BE070030A30023080318230FBF072308E4
:101C00000318230FC0070310670C8316A00083126C
:101C10003E088316A10083123F088316A200831298
:101C200040088316A3002008A10700308312A300F8
:101C3000831622088312A2000318230F230783169A
:101C4000A20023088312A2000318230F2307831680
:101C5000A30021088312A100831622088312A20088
:101C6000831623088312A3006308A400A501A6011C
:101C70008A11042083122708BE002808BF00290803
:101C8000C0008A156C1E4B2E3E08BB003F08BC00EE
:101C90004008BD006C12C7208A155E2083125508CB
:101CA000A100A201A301A030A4008630A50001304C
:101CB000A6008A110420831227088316A00083122D
:101CC00028088316A100831229088316A200831214
:101CD0005608A100A201A3011030A4002730A500DE
:101CE000A6018A110420831227088316A3008312F9
:101CF00028088316A400831229088316A50020084B
:101D0000A6002108A7002208A8002308A607240887
:101D10000318240FA70725080318250FA807831207
:101D20005708A100A201A301E830A4000330A500D8
:101D3000A6018A110420831227088316A9008312A2
:101D400028088316AA00831229088316AB002608E8
:101D5000AC002708AD002808AE002908AC072A0807
:101D600003182A0FAD072B0803182B0FAE07831299
:101D70005808A100A201A3016430A400A501A60196
:101D80008A110420831227088316AF0083122808C3
:101D90008316B000831229088316B1002C08B20004
:101DA0002D08B3002E08B4002F08B207300803181E
:101DB000300FB30731080318310FB40783125908E5
:101DC000A100A201A3010A30A400A501A6018A1165
:101DD0000420831227088316B5008312280883166F
:101DE000B600831229088316B7003208B8003308FA
:101DF000B9003408BA003508B80736080318360F9A
:101E0000B90737080318370FBA0738088312E900F3
:101E1000831639088312EA0083163A088312EB000E
:101E20005A08E9070030A30023080318230FEA0724
:101E300023080318230FEB076908A1006A08A20012
:101E40006B08A3006308A400A501A6018A11042061
:101E500083122708E9002808EA002908EB003E0859
:101E6000E9023F08031C3F0FEA024008031C400F31
:101E7000EB02A2016B0822028A15031D452F6A0896
:101E80002202031D452F690867020319922F0318C8
:101E9000922F6708E902A2012208031C220FEA021E
:101EA0002208031C220FEB02A2016B082202031D71
:101EB0005F2F6A082202031D5F2F69086802031959
:101EC000802F0318802F6808BE070030A300230866
:101ED0000318230FBF0723080318230FC007C720C9
:101EE0008A155E2083126808E902A2012208031CF9
:101EF000220FEA022208031C220FEB028A15542F3C
:101F000069086A046B040319922F6908BE076A08FE
:101F100003186A0FBF076B0803186B0FC007C720B1
:081F20008A155E208A154C2988
:02400E00023D71
:00000001FF
